S10E24008E0FFFBD27864FCE20008CFE
S111240B20082705A7000820F6CE278D18CE3E
S111241920008C278D270AE60018E70008181B
S11124270820F1CC0000270CC320083736CC67
S10E24352008BD274138BD244020FED4
S1112440BD26DC04C63EF710097F2005C6FF4A
S110244EF72004CC003CBD24AECC000CBD36
S111245B24AECC0006BD24AECC0001BD24AEE0
S1102469CC0080BD24AECC26B8BD24E9CC47
S111247600C0BD24AECC26ADBD24E9CC00943C
S1102484BD24AEBD25A9ED026D0327F7F6BA
S111249120054F5D2A0143BD24CB20EA8FC3F2
S111249F00048F353839F6B5F0C4805D26F898
S11024AD3937363C3C30EF00EC04E705BD48
S11124BA24A5E605F7B5F08FC300028F353870
S11124C818383937363C3C30EF00BD24A5E609
S11124D6054F5D2A0143F7B5F18FC300028F55
S11124E4353818383937363C3C30EF002015B7
S11124F21AEE0418E6004F5D2A0143BD24CB08
S1112500EC04C30001ED041AEE04186D00266D
S111250EE38FC300028F3538183839BD26DC40
S110251C46EC08272BCC0000ED02201DCC5E
S11125290000ED042007EC04C30001ED04ECF7
S1112537041A83004925F1EC02C30001ED02F1
S1112545EC021AA30823DC8FC300068F35387E
S1112553183839BD26DC46EC082731CC0000D0
S1112561ED022023CC0000ED04200DCC00017F
S111256FBD2519EC04C30001ED04EC041A832D
S111257D006425EBEC02C30001ED02EC021A2F
S111258BA30823D68FC300068F3538183839BD
S11125993132334134353642373839432A3033
S10525A72344C7
S11125A9BD26DC14EC00C3000418CE25993CBA
S11125B78FCC0010BD26C4387F2003C604F765
S10F25C520027E265CF62002F71008BD00
S11125D1267EF6100AF7200118CE2001181DF0
S11125DF00F07D20012764F62001C1042605CA
S11125EDC603F72001F62001C1082605C60426
S11125FBF72001F620014F830001F720014F65
S1112609ED02F620034FE302F72000F1200457
S1112617260BCC00008FC300148F353839F623
S11026252000F72004EC00C30004ED02F6D1
S111263220004FE302188F18E600F72005CCB5
S111264000018FC300148F353839F620024F85
S111264E05F72002F620034FC30004F7200313
S110265CF62002C14024037E25CAC6FFF704
S11126692004CC00008FC300148F3538398F45
S1102677C300148F353839CC00003939BD4B
S111268426DC042003BD267EBD25A9ED026DD3
S11026920327F4F620054F5D2A01438FC392
S111269F00048F3538398FC300048F35383965
S11126AD5072657373204B657973004B657929
S10C26BB7061642054657374001D
S11126C41A83000027113718E600E70033835D
S10D26D20001270508180820EF395D
S11126DC1838181F00400237363C3018E6004C
S11126EA4FC43F37368F30A3008F35EF0018F2
S11126F81F0080043C3C3C3C186E0118303737
S111270636188FC30001183018EE0218EB00CD
S11127148900188F3233183C183018AE0018A4
S1082722EE02186E0137
S111272737363C303C30EC04F7102BC60CF770
S10F2735102D8FC300028F35381838397E
S1112741BD26DC46EC08ED041AEE04FC20066E
S111274F18ED00EC04FD2006EC08C30006EDB6
S111275D02EC0CA3023736EC04C30004188F00
S111276B323318ED00EC04C30002188FEC0C9E
S110277918ED008FC300068F35381838396D
S10A2786CC0030BD27273908
S9032400D8
